S31508001800000A0020D9180008E7180008E918000897
S3150800181000000000000000000000000000000000BA
S315080018200000000000000000000000000119000888
S3150800183000000000000000000319000855370008E2
S3150800184001420008071900080719000807190008C7
S3150800185007190008071900080719000807190008DA
S31508001860071900089528000807190008071900082D
S3150800187007190008071900080719000807190008BA
S3150800188007190008000000000000000007190008FA
S3150800189000000000071900080719000807190008C2
S315080018A00000000007190008071900084D3C000849
S315080018B007190008071900080719000800000000A2
S315080018C0EE11AA550348854600F0B2FC00480047C9
S315080018D0FD4F0008000A00200B4880F308880B48D3
S315080018E080470B480047FEE704207146084202D0AD
S315080018F0EFF3098001E0EFF30880714603F07EFA02
S31508001900FEE7FEE7FEE7FEE7000A00209D3800082E
S31508001910C518000830B50B460146002020220124D0
S3150800192009E00D46D5409D4205D31D469540491B05
S315080019302546954040191546521E002DF1DC30BD4E
S3150800194070B500242546002801DA01244042002902
S3150800195001DA01254942FFF7DDFFAC4200D04042DB
S31508001960002C00D0494270BD03460B439B0703D0A9
S3150800197009E008C9121F08C0042AFAD203E00B7846
S315080019800370401C491C521EF9D27047D2B201E0BE
S315080019900270401C491EFBD270470022F6E710B5BC
S315080019A013460A4604461946FFF7F0FF204610BDBF
S315080019B0F8B502464A40D40F42004B0052085B086D
S315080019C09A4202D20246084611464A0023D0C30D5F
S315080019D04A00DDB2120EAD1A202D35DA490201266B
S315080019E0490AF6058A19002C00D0524220214F1BBD
S315080019F01146B9402A411018C20D9A4221D0002C2E
S31508001A0017D0012D08DCDA05801AD20F8019D20703
S31508001A10DBB200F023FBF8BDDA05801A012340008B
S31508001A201B06C01880185A428018CA0F104349006E
S31508001A3007E04908C2071143DA05801A80194008E9
S31508001A40801800F003FBF8BD61000122511A001B43
S31508001A50F7E70122D2075140AAE70122D2075040F0
S31508001A60A6E7024670B54A40D30FDB0740002DD0E3
S31508001A704A002AD0010E140E000212020919400A61
S31508001A80520A8418E50104465443000A120A2E0431
S31508001A905043A4194219200CC543AA18120C012553
S31508001AA0AD03521C521912047F39240400D0521C6B
S31508001AB0104301D44000491EC2B20C06C0092018C2
S31508001AC0401C4008802A02D003E0002070BD400870
S31508001AD04000002900DA0020184370BD70B50246A0
S31508001AE04A40D50F40004A00ED0740085208002832
S31508001AF014D0002A12D0C40DD30D41020120C0050E
S31508001B005202490A520AE41A091812187D349142F7
S31508001B1001D3641C00E04900002C01DA002070BDE6
S31508001B200023914201D3891A03434008490000283B
S31508001B30F7D100290AD0914202D10121C90705E04F
S31508001B40914201D2012101E00121C943E005C018F3
S31508001B50401900F07BFA70BDF0B5074608465840B4
S31508001B6087B0C00F049048000E465900400849083F
S31508001B70BC1A884105D2384631461E4617460B46DA
S31508001B8002465800400810434CD0300D03904005DB
S31508001B905900400D490D0590401A0290402872DA06
S31508001BA018030121000B09050843019004980092C7
S31508001BB0002805D0019952420020884100920190E0
S31508001BC0029840210A1A0199009800F00BFA054676
S31508001BD00C466B4607CB00F026FAC0197141039AEA
S31508001BE00E0D0023D71756401A467A40164344D09E
S31508001BF0049A002A2DD0029A012A039A15DC1205A6
S31508001C00C01A914101263605001C7141D20F059E66
S31508001C10D2070093019202962A46234600F064FAF8
S31508001C2007B0F0BD38463146FAE71605224A0F4690
S31508001C30B218C01AB74101210905001C4F41001806
S31508001C407F41114618187941E20F10436D19644116
S31508001C5013E0E2076D0815436408C2071443039AA4
S31508001C6001261205C01A91413605001C7141CE079E
S31508001C70400830434908C01851412A46234600F017
S31508001C8026FACDE7FFE7049801224000C117121A89
S31508001C9000238B4104983146C417381AA141EEE750
S31508001CA030B40124E407634030BC55E730B401245E
S31508001CB0E407614030BC4FE70000E0FFF0B51FB411
S31508001CC088B00B990998002448400999C00F490023
S31508001CD049080991C0070B990090490049080B91DA
S31508001CE009990898A64608431CD00B990A980843F0
S31508001CF018D0099801244000420D4800410D099862
S31508001D0024050003000B204309900B980003000BE1
S31508001D1020430B9050181C49401800220190144685
S31508001D20104605E0002001460DB0F0BD032801DA93
S31508001D30034600E003239C46C11A0AAE0AE05F0088
S31508001D4008ADED5B4F00F75B7D430027AA187C4181
S31508001D50491C5B1E6145F2DD410004AB5A52210461
S31508001D60120C0A43240C401C0828DFDB0198029059
S31508001D700099704601910090059B049A0799069868
S31508001D8000F0B2F9D0E700000DFCFFFFF0B50C46F5
S31508001D905C4085B0E40FE40703944C000026640811
S31508001DA059009446490802460296224321D06246C3
S31508001DB00A431ED06200570D4A000E032303550D31
S31508001DC0012402462C492405781B1B0B360B4018A8
S31508001DD023432643614600901C46501AB44103D358
S31508001DE00098401C009002E0921800985B41002879
S31508001DF003DA0020014605B0F0BD002001210905DF
S31508001E000746864611E064461D46141BB54106D3AF
S31508001E106546521BB341744607430C43A646CD0795
S31508001E2040084908284392185B4105460D43EAD104
S31508001E301046184313D0604619465040714008436F
S31508001E4006D06046101AB34106D20122002306E0E6
S31508001E5000220123DB0702E00122D2435310009837
S31508001E6074460105381C6141029C039D00196941AD
S31508001E7000F02DF9BFE70000FD030000C217C10FEF
S31508001E80504010B54018CA079623002100F0E6F81E
S31508001E9010BD10B500229623114600F0DFF810BDDC
S31508001EA00EB5C217C10F5040CA0740180021054B8E
S31508001EB00293019200910A460B4600F015F903B009
S31508001EC000BD0000330400000EB50549029100214B
S31508001ED000910A460B46019100F006F903B000BDD1
S31508001EE033040000410040020122400AD205090ECF
S31508001EF080187F2901DA00207047962903DC96228C
S31508001F00511AC84070479639884070474A000903F5
S31508001F100123090B1B051943094B10B5520D9A42AB
S31508001F2001DA002010BD064B34339A4203DC9A1AB4
S31508001F3000F068F810BD03495118884010BD00002C
S31508001F40FF030000CDFBFFFFC20FD2074000400889
S31508001F500BD0C10D0723DB01C91840020905400A49
S31508001F601143C208400711437047002001467047D5
S31508001F7010B5002904DB0124E40740428C412146C0
S31508001F80002B04DB1C460123DB075242A3418B428C
S31508001F9000D1824210BD0000CB0FDB07490010B507
S31508001FA0490802460A4307D00A0D07240903E40133
S31508001FB0090B121B002A01DC002010BDC900440FC2
S31508001FC00C43C100E018D205801800F03FF810BD98
S31508001FD00122D207002800DB101A002900DB511A5B
S31508001FE08142704710B5202A04DB0146203A914009
S31508001FF0002010BD914020239C1A0346E340194354
S31508002000904010BD10B5202A04DB0846203AD0407F
S31508002010002110BD0B46D340D0402024A21A91407F
S315080020200843194610BD10B5202A06DBCB1708460B
S31508002030203A1041C1170B4306E00B461341D04026
S315080020402024A21A91400843194610BD002904DA33
S31508002050401C490001D140084000704770B4002474
S31508002060050C05D11024000402D1002921D0112421
S31508002070050E01D100020834050F01D10001241D07
S31508002080850F01D18000A41C002801DB4000641CD8
S31508002090002908D020252E1B0D46F540A14000D06A
S315080020A001212943084301061B1B000ADB1D02D533
S315080020B0002070BC7047DB05181880180029F8DA6C
S315080020C0401C4900F5D170BC40084000704710B567
S315080020D0002B08DA0024401C614192185B411A4320
S315080020E001D14008400010BDF0B51FB482B00546C6
S315080020F00C0003D0084602F0E9F802E002F0E6F820
S3150800210020300246009021462846FFF76BFF049BC5
S31508002110059A04460F4618431143084314D0184637
S3150800212010431BD0009840210A1A18460599FFF754
S3150800213069FF05460E46009A05990498FFF752FF6F
S31508002140084305D0012004E02046394607B0F0BD13
S315080021500020C11705430E432C43374300990E98B8
S315080021606305401A7905E40A00220C43FD0A0A3081
S3150800217002D500200146E9E70105101969410C9CC2
S315080021800D9D00196941FFF7A2FFDFE7FEB50023A1
S315080021901A461B1A8A4103DB0020014603B0F0BD2C
S315080021A04A000D0301212D0B0905520D0D43D107D8
S315080021B002D100186D41521E5110FF31FF31013115
S315080021C0002704463E4638460097019102460121FB
S315080021D000200905FFF716FFC3197141F8183246A2
S315080021E084468E464A4161462846611A904104D380
S315080021F06046241A954176461F46241900986D4173
S31508002200401C00903428E1DDF91930467041091B5D
S31508002210A84103D20022D243134601E00022134606
S3150800222001980105381C7141FFF751FFB6E7000018
S31508002230064C0125064E05E0E36807CC2B430C3C0B
S3150800224098471034B442F7D3FFF740FBAC65000853
S31508002250CC65000810B50446002C08D101210920D8
S31508002260C00600F0E3FD002000F0E6F852E0012C7D
S3150800227005D102210920C00600F0D8FD4AE0022C4B
S3150800228005D104210920C00600F0D0FD42E0032C48
S3150800229005D108210920C00600F0C8FD3AE0042C43
S315080022A005D110210920C00600F0C0FD32E0052C3A
S315080022B005D120210920C00600F0B8FD2AE0062C29
S315080022C005D140210920C00600F0B0FD22E0072C08
S315080022D005D180210920C00600F0A8FD1AE0082CC7
S315080022E004D101210D4800F0A1FD13E0092C04D109
S315080022F002210A4800F09AFD0CE00B2C04D11021AB
S31508002300064800F093FD05E00C2C03D18021034814
S3150800231000F08CFD204600F08FF810BD0004004840
S315080023207FB500200090019002900390002427E0DA
S3150800233000250CE0E800294940186100405AA10030
S315080023406A4651584018A1005050681C85B2142D91
S31508002350F0DBA1006A4650581421FFF7DBFA282162
S31508002360484361001E4A515A3C225143461864218B
S315080023703046FFF7CFFA6100194A5052601C84B202
S31508002380042CD5DB1748C078002826D01448408886
S315080023901549884203DC1248808888420ADD1148BC
S315080023A02038C079002805D11049486001210D4818
S315080023B02038C1710A4840880A2803DB0848808803
S315080023C00A280ADA07482038C079002805D10749BB
S315080023D04860012103482038C1717FBD44040020AC
S315080023E03C010020C4030020E60F0000C4010020C1
S315080023F000B587B001A800F0AFF80121480201F046
S315080024001BF80020019070200290012080020390A2
S3150800241000200690059001A9064800F031F8012130
S31508002420044800F021F80121024800F011F807B02D
S3150800243000BD00000024014010B504460723002211
S315080024402146024800F038F810BD0000002401407B
S31508002450002904D0426801231A43426003E0426817
S315080024605208520042607047002904D08268082347
S315080024701A43826003E0826808239A4382607047A1
S3150800248042680B4B1A4042600B684A681A43436815
S315080024901A4342608268074B1A4082600B694A6990
S315080024A01A438B681A4383681A4382607047000090
S315080024B00FBCFFFF8FF1F9FFF0B504460D4616462F
S315080024C01F463F073F0F2B46082B0FD91B071B0F2D
S315080024D0083B606F9A000F21914088436067606FE0
S315080024E099003A468A40104360670BE0206F9A00CD
S315080024F00F21914088432067206F99003A468A4009
S3150800250010432067E0680121A9408843E060E0683D
S315080025100121A9400843E0600120800328400028E3
S3150800252003D0012000F020F807E00120C00328406E
S31508002530002802D0012000F017F8F0BD002905D0C8
S315080025408268FF2301331A43826004E08268FF230E
S3150800255001339A43826070470021016041608160BF
S315080025600173016141617047002806D00649496830
S315080025700C221143044A516005E0034949680C22BC
S315080025809143014A516070470024014010B5244820
S315080025900078012834D10020214908702149088093
S315080025A012E02048008840001F49085A1F49098838
S315080025B0C9001F4A89181B4A1288520088521948AE
S315080025C00088401C17490880164800880428E8DB5C
S315080025D07E2001F021FE022000F02EF90121154887
S315080025E0FFF7ACFF11480088401C104908800846D0
S315080025F00088142804DB0020088001200E49087092
S315080026000D480078002806D0FFF78AFE00200A4900
S31508002610087000F055FC7E2001F0FEFD10BD00009C
S315080026204C010020660100200C04002068010020EF
S31508002630440400200024014044010020FFB583B073
S315080026400C46029400200190002726E000261CE094
S31508002650721C039951430846791CFFF75BF9054636
S31508002660A54201D9281B00E0601B05460298A8422E
S3150800267004D90295059806700698077002980028EE
S3150800268002D10120019002E0761C402EE0D300BF63
S315080026900198002800D002E07F1C042FD6D300BF83
S315080026A0029807B0F0BD000000BF00BF00BF00BF22
S315080026B000BFBFF34F8F00BF00BF00BF06480749E2
S315080026C0C86000BF00BF00BFBFF34F8F00BF00BF89
S315080026D000BF00BF00BFFDE70400FA0500ED00E0FB
S315080026E010B500F001F810BD10B523480078002891
S315080026F017D1224800F028FF01283CD11F4800784E
S31508002700002838DD1D480078402834DC01F071FACD
S315080027101B490860012018490870002019490870EB
S3150800272029E0164A17490978491C501800F00CFF89
S31508002730012816D113480078401C124908700F4822
S3150800274000780978884216D100200B4908700B4892
S315080027504078FF280FD10B48007802280BD1FFF7E5
S31508002760A3FF01F046FA064909686431884202D98E
S3150800277000200149087010BD15010020C80300207B
S31508002780180100201401002010B586B00446012166
S31508002790880300F051FE0121480400F02DFE0122B5
S315080027A00921C80600F02DFB01220A210920C006CE
S315080027B000F027FB01A801F022FB019430216846AE
S315080027C0018100214181818101821821C18101A9EC
S315080027D0184801F0D1FA0121164801F0AAFA05A80D
S315080027E000F065FB01214902684681820121817555
S315080027F01821C17505A90920C00600F0B5FA0121FE
S315080028008902684681824821C17505A90920C00642
S3150800281000F0AAFA1B2168460170032141700121C4
S31508002820817000F0B5FD01220221024801F099FAF3
S3150800283006B010BD0038014001B50449009808608B
S3150800284000BF024800680028FBD108BD1C01002013
S31508002850014600220E4B1A61CA005A6100229A618B
S3150800286005221A6100BF0A4A1069C207D20F002A58
S3150800287004D0012212040240002AF4D0044A126944
S3150800288052085200024B1A6100229A6170470000F2
S3150800289000E000E010B500210448FFF74FFE0220D3
S315080028A000F04AF801200249087010BD00240140D2
S315080028B04C01002000B589B00121084600F09CFDB6
S315080028C01A4800F045F801A800F08EF8184801905B
S315080028D0184802900021684601730420049068464F
S315080028E00175802141754900C18289000183202133
S315080028F08176090281830021C183018401A90B48DD
S3150800290000F04CF80121094800F01CF801220221C8
S31508002910064800F039F8092168460170022141701D
S315080029200121817000F034FD09B000BD08000240A5
S31508002930002401400C04002001494860704700004B
S31508002940000002400268520852000A4302607047BB
S3150800295010B504462068400840002060002020602A
S315080029606060A060E060E1B2084608380521FEF71D
S31508002970D1FF01460F2088400249496808430149AA
S31508002980486010BD00000240002A03D003680B43CC
S31508002990036002E003688B430360704710B50A7A48
S315080029A08B7D1A430B7C1A434B7C1A434B8A1A437A
S315080029B08B8A1A430B8B1A434B8B1A430368094CB1
S315080029C023401A43026002680123DB039A438B8B78
S315080029D01A430260CA6842600A6882604A68C2602E
S315080029E010BD00000F80FFFF0021016041600172E9
S315080029F0C16001744174418281828175018341837A
S31508002A008183704770B506460C4621460A4800F091
S31508002A104BF90546002D01D1401E70BD064885427A
S31508002A2002D10648051B00E02D1B224629463046E2
S31508002A30FEF79AFF2046F0E700F4000800FC0008BD
S31508002A4070B506460C4621460A4800F02DF905469B
S31508002A50002D01D1401E70BD0648854202D10648A8
S31508002A60051B00E02D1B224629463046FEF77CFF53
S31508002A702046F0E7008000080088000870B5064682
S31508002A800C4621460A4800F00FF90546002D01D1EB
S31508002A90401E70BD0648854202D10648051B00E067
S31508002AA02D1B224629463046FEF75EFF2046F0E7F4
S31508002AB0009000080098000870B505460C462246A6
S31508002AC00249284600F0B1F8204670BD00F4000817
S31508002AD070B505460C4622460249284600F0A5F878
S31508002AE0204670BD0080000810B5044608480069F5
S31508002AF002210843064908610846446100694021E5
S31508002B00084303490861034800F00EF910BD0000A8
S31508002B1000200240FF0F00000C48C068C007C00F25
S31508002B20002801D0012070470848C06804210840E1
S31508002B30002801D00220F6E70448C06810210840A2
S31508002B40002801D00320EEE70420ECE7002002402D
S31508002B50034800698021084301490861704700005D
S31508002B600020024030B504460D460548006901219B
S31508002B7008430349086125800F2000F0D5F830BDC9
S31508002B800020024010B57E2001F046FB064800F002
S31508002B900FF87E2001F040FB044800F009F87E207B
S31508002BA001F03AFB10BD000000F4000800800008A0
S31508002BB010B5044600F0ACF82046FFF795FFFFF77E
S31508002BC0C7FF10BD70B503460125002208E0500076
S31508002BD01C5A0748844201D0002506E0501C82B2E0
S31508002BE0CE0F761876109642F1DC00BF284670BDE7
S31508002BF0FFFF0000F8B505460E46144600F088F8B3
S31508002C007E2001F009FB002707E029883046FFF7F8
S31508002C10A9FFB61CAD1C781C87B2E10F091949102B
S31508002C20B942F2DCFFF794FFF8BDF8B507460C4643
S31508002C3015462946204600F037F80646002E0DD1DF
S31508002C402046FFF7B5FF012080022018FFF7B0FFE6
S31508002C502A4621463846FFF7CDFF24E001208002A8
S31508002C602018401BB0420AD1012080022018FFF725
S31508002C709FFF2A4631463846FFF7BCFF13E001207E
S31508002C80C0022018401BB04208D12046FFF790FF2B
S31508002C902A4631463846FFF7ADFF04E02A46314654
S31508002CA03846FFF7A7FFF8BDF8B505460E462F4686
S31508002CB0E807C00F002801D000BFFEE73146012013
S31508002CC0C002FEF73DFE002901D000BFFEE7002442
S31508002CD00BE020467043471931463846FFF772FF26
S31508002CE0012800D108E0601C84B231460120C002E8
S31508002CF0FEF726FEA042ECDC00BF31460120C002EA
S31508002D00FEF71EFEA04200D100273846F8BD000097
S31508002D1002480349486003484860704723016745ED
S31508002D2000200240AB89EFCD10B5024600BFFFF781
S31508002D30F3FE0346521EFF2400E0641E002CFCD15D
S31508002D40012B01D1002AF2D1064800697721884370
S31508002D50044908613420C860002A01D1052010BD45
S31508002D601846FCE700200240F8B50246CD782F0742
S31508002D703F0FCD7810263540002D01D08D782F4392
S31508002D801446002011E085062B0E0D880126864084
S31508002D903540002D07D025680F269E40B5433E4690
S31508002DA09E4035432560451CE8B20828EBDB141D18
S31508002DB00D882D120095002011E085062B0E0125A1
S31508002DC08540009E3540002D07D025680F269E4079
S31508002DD0B5433E469E4035432560451CE8B2082863
S31508002DE0EBDBCD78282D04D155690E88354355611E
S31508002DF006E0CD78482D03D115690E88354315614F
S31508002E00F8BD70B54D07EB0E082902DA05462035E0
S31508002E1001E0054624352C460F269E402568B54315
S31508002E2016469E403543256070BD000038B50446F9
S31508002E300D460920C006844203D10121480400F04A
S31508002E40DBFA1148844203D10121000200F0D4FACA
S31508002E500E48844203D10121000200F0CDFA0C4845
S31508002E60844203D10121080500F0C6FA684600F03D
S31508002E701EF868460580012181700021C1706946E7
S31508002E802046FFF771FF38BD0004004800080048D7
S31508002E90000C0048024690680840002801D001202E
S31508002EA070470020FCE741617047016170470021C7
S31508002EB0C9430180022181700421C1707047000056
S31508002EC0F0B58FB00025002600200D900C907E20CE
S31508002ED001F0A2F900241AE06100A94A505AFEF747
S31508002EE0D8FFA8490790FEF7F9FD0746FFF72CF823
S31508002EF00022A54B09910890FEF7E0FE0B910A9077
S31508002F00FFF74AF8A100A14A5050601C84B2042C6D
S31508002F10E2DB9E498868FFF717F89D4A9D4B0591A5
S31508002F200490FEF7BDFE00229B4B07910690FEF724
S31508002F302DFF9A4A9A4B09910890FEF7B7FE0B9116
S31508002F400A90FFF729F8054690494868FEF7FCFFFE
S31508002F508F4A904B05910490FEF7A2FE00228E4BF5
S31508002F6007910690FEF712FF8C4A8D4B099108903F
S31508002F70FEF79CFE0B910A90FFF70EF806462846C8
S31508002F80FEF7E2FF0022874B05910490FEF78EFEBE
S31508002F900991089029468448FEF763FD0746FEF71F
S31508002FA0D3FF07910690099B089AFEF7EFFE0B914F
S31508002FB00A90FEF7F1FF7D4908603046FEF7C4FF28
S31508002FC00022784B05910490FEF770FE099108904F
S31508002FD031467548FEF745FD0746FEF7B5FF0791EA
S31508002FE00690099B089AFEF7D1FE0B910A90FEF708
S31508002FF0D3FF6F4908606F49088BFEF765FF6E4A75
S315080030006E4B03910290FEF759FE00226C4B059118
S315080030100490FEF7BBFE099108906649088BFEF7F7
S3150800302038FF0746FEF790FF0022654B0191009096
S31508003030FEF7ACFE059104905C480068FEF784FF35
S3150800304003910290059B049AFEF72AFE07910690C3
S31508003050099B089AFEF79AFE0B910A90FEF79CFFC9
S315080030600D905449488BFEF72FFF534A534B039153
S315080030700290FEF723FE0022514B05910490FEF7BD
S3150800308085FE099108904B49488BFEF702FF0746D3
S31508003090FEF75AFF00224A4B01910090FEF776FE92
S315080030A00591049042480068FEF74EFF039102908E
S315080030B0059B049AFEF7F4FD07910690099B089A6A
S315080030C0FEF764FE0B910A90FEF766FF0C903D48EA
S315080030D00D99FEF76DFC0746FEF704FF3A490860AE
S315080030E038480C99FEF764FC0746FEF7FBFE37499D
S315080030F008603748008A344909684018C003010C3B
S3150800310033480182408A314909684018C003010CD6
S315080031102F4841821D49C8682E49FEF7A2FC07467A
S31508003120FEF7E0FE81B22A480184FF38C1380088DC
S31508003130FF21F531884220DD00201E4950390880DC
S31508003140124908682449FEF743FF11D22048203067
S31508003150C079002806D117495039486001211C4812
S315080031602030C171FF2101311C48FFF79EFE04E0A3
S31508003170FF2101311948FFF796FE0FB0F0BD000098
S315080031803C01002000F07F45000008403404002080
S31508003190333333333333C33F000028404A0C022B02
S315080031A08716D13F00000440000048435401002020
S315080031B05801002014020020091B9E5E29CB703F8F
S315080031C000408F400000C8415C01002060010020DB
S315080031D0840300200000C8427B142E3F00040048E8
S315080031E00148006870470000200100200348006875
S315080031F003490978401801490860704720010020F2
S315080032002801002008B50121480400F0F5F801213D
S31508003210880400F0F1F86846FFF749FE0121C90362
S31508003220684601804821C17069460920C006FFF733
S315080032309BFD6846FFF73BFE0121090368460180AE
S315080032404821C17069460920C006FFF78DFD68460A
S31508003250FFF72DFE4021684601800421C1706946AA
S315080032600148FFF781FD08BD0004004810B501219B
S31508003270C9030920C006FFF70DFE002808D1234818
S31508003280807A002808D1012120488172817103E0E3
S3150800329000211E48817181721D4880681D49884237
S315080032A02DD900201A4988600021184881712030DC
S315080032B0C07800281DD108211748FFF7F6FD1348E6
S315080032C09038408803280CDA10482038408A82282B
S315080032D004DA01210D482030C17002E001210B48B3
S315080032E0C1710A484079012809D100200849486077
S315080032F005E00020064948600021044841717E2007
S3150800330000F08AFF0148807910BD0000A403002060
S31508003310C4010020DC0500000004004808B50121AE
S31508003320480400F069F80121880400F065F8684649
S31508003330FFF7BDFDFF212A31684601800121817012
S315080033401021C17069461148FFF70EFDB62168467F
S315080033500180012181701021C17069460920C006CB
S31508003360FFF702FD10210920C006FFF79CFD80210A
S315080033700920C006FFF797FD01210448FFF793FDD2
S3150800338008210248FFF791FD08BD00000004004827
S315080033908178002925D01749032212028918027854
S315080033A092109200895802789207D30EFF229A400B
S315080033B0914342789207120E03789B07DB0E9A40D8
S315080033C011430C4A03231B02D21803789B109B0057
S315080033D0D1500178CA06D20E01219140054A1160E2
S315080033E007E00178CA06D20E01219140014A8032CF
S315080033F01160704700E100E0002905D0054A5269CE
S315080034000243044B5A6104E0024A52698243014B63
S315080034105A61704700100240002905D0054AD26952
S315080034200243044BDA6104E0024AD2698243014B43
S31508003430DA61704700100240002905D0054A9269F2
S315080034400243044B9A6104E0024A92698243014BA3
S315080034509A6170470010024010B500F031F804492F
S315080034604968F02211400909024A515CC84010BD5A
S3150800347000100240EE00002010B5FFF7EDFF0549E9
S315080034804968072212021140090A034A515CC840DA
S3150800349010BD000000100240EE00002010B5FFF736
S315080034A0DBFF054949680722D2021140C90A034AC7
S315080034B0515CC84010BD000000100240EE0000201C
S315080034C0F8B51E4840680C210840042802D0082890
S315080034D02ED101E01A4C2DE0184840300069C0078B
S315080034E0C00F00280AD0154840300069022108405C
S315080034F0002801D0134802E0114800E010480746AA
S315080035000E4840300069FF2109040840000C451C9C
S315080035100A4840300069072109020840000A461C8B
S315080035203946694308463146FEF7F4F9044601E090
S31508003530034C00BF00BF2046F8BD00000010024043
S3150800354000127A0000093D0070B5044600250221E4
S31508003550074800F0F4FB002808D0054800F048FCAE
S3150800356020700221024800F0E2FB0125284670BDC2
S315080035700038014010B500F001F810BD00B585B05F
S3150800358062480068012108436049086000BF5F4837
S315080035900068022108400028F9D05D485D490860A6
S315080035A05D480068102108435B49086008460068C2
S315080035B0C008C000086057490968481E5749FEF701
S315080035C0A9F904905448006804994907490F084323
S315080035D0514908604D484068514908404B49486080
S315080035E008464068902108434849486008464068AC
S315080035F04860484800684649884207D943484068B1
S31508003600052109020843414948600BE04148006822
S315080036104449884206D93D48406801218902084341
S315080036203A4948606B4601AA3A4801683E48FFF79E
S3150800363005F8364840300069800880003349403133
S315080036400861084600694008400008616846007835
S315080036504007400F0290684600794006400E0390E6
S315080036602A48C069890508432849C861274840305F
S3150800367000692E490840254940310861039800042D
S3150800368002990902084321494031096908431F493B
S31508003690403108611D4800680121090608431B4995
S315080036A0086000E000BF1948006801214906084083
S315080036B00028F7D0154840688008800013494860FC
S315080036C008464068022108431049486000E000BFE8
S315080036D00E4840680C2108400828F8D10120FFF759
S315080036E0B7F80A484068102188430849486001200D
S315080036F0FFF7AEF8054840688021884303494860CB
S315080037000120FFF7A5F805B000BD00000010024033
S3150800371000A24A04000100200020024000366E0183
S315080037200FC0FFFF0051250200127A00FFF800FFC4
S31508003730042806D10649096904221143044A11617D
S3150800374005E00349096904229143014A116170475A
S3150800375000E000E010B5FFF749FD4D480088401C21
S315080037604B49088008464068401C4860494800683C
S31508003770002804D047480068401E46490860464865
S315080037808079012805D142488068401C40498860F4
S3150800379002E000203E4988603F48C078012805D1EC
S315080037A03B480069401C3A49086102E00020384954
S315080037B008613948007A012805D13548C06B401C94
S315080037C03349C86302E000203149C8633049486874
S315080037D00A21FEF79FF800291CD12F48C17F807F58
S315080037E0814206DD2C48807F401CC1B22A48817779
S315080037F010E02948C17F807F814200D10AE026482F
S31508003800C17F807F814205DA2348807F401EC1B28E
S315080038102148817720482030C078022804D01E48E5
S315080038202030C078032804D11948406B401C184939
S31508003830486319482030407800280AD116482030B5
S31508003840C078042805D11248406C401C10494864C9
S3150800385002E000200E4948640F48C07A012805D1C5
S315080038600B48C06C401C0A49C86402E0002008499D
S31508003870C8640948007B012805D10548806C401CAE
S315080038800349886402E000200149886410BD0000ED
S31508003890C40100201C010020A403002010B516480E
S315080038A0006801210843144908600846406813491E
S315080038B008401149486008460068114908400E4901
S315080038C00860084600680121890488430A49086097
S315080038D008464068C32109048843074948600846E2
S315080038E0006808490840044908609F200004886069
S315080038F0FFF740FE10BD0000001002400CC0FFF8A4
S31508003900FFFFF6FEFFFF8F0008B501214804FFF709
S3150800391073FD022201210920C006FFF772FA02216F
S31508003920684601801821C170012181706946092005
S31508003930C006FFF719FA01214804FFF75DFD0222C8
S3150800394011460920C006FFF75CFA04216846018083
S315080039501821C1700121817069460920C006FFF748
S3150800396003FA08BD30B587B004460D46012108465E
S31508003970FFF752FD04A800F033F90594684605825E
S31508003980002101838176817404A90120800700F053
S31508003990F1F8684600F0D2F8602168460170012106
S315080039A04170002001900021684601726946012095
S315080039B0800700F057F869460120800700F08AF86A
S315080039C00821C80600F07EF80821C80600F0B0F8FD
S315080039D04021080600F038F84021080600F03CF8B7
S315080039E00121880700F00AF80121880700F01EF86F
S315080039F00121880700F00EF807B030BD002904D071
S31508003A00026880231A43026003E0026880239A430F
S31508003A1002607047002904D0026801231A43026035
S31508003A2003E002685208520002607047002905D078
S31508003A30426C0123DB031A43426404E0426C01230F
S31508003A40DB039A4342647047826907231B039A4340
S31508003A500B021A4382617047C26970239A430A436C
S31508003A60C261704710B5826907231B039A430B7816
S31508003A701B021A4382610A7A12014B781B011A4308
S31508003A80036A3024A3431A4302624A6882630C4AD3
S31508003A90904213D14A7A12018B781B011A43036AA2
S31508003AA0C024A3431A4302624A8992008B899B0069
S31508003AB01A4343682401A3431A43426010BD000019
S31508003AC0002C014082690123DB029A430B021A4348
S31508003AD08261704710B5C26970239A430B781A43FE
S31508003AE0C2610A7A12024B781B021A43036A03243C
S31508003AF02402A3431A4302624A68C2630B4A9042ED
S31508003B0013D14A7A12028B781B021A43036AA4005D
S31508003B10A3431A4302624A8912018B891B011A437D
S31508003B204368A400A3431A43426010BD002C014019
S31508003B30C26908239A430A43C2617047002101708B
S31508003B404170817041600172417241818181704783
S31508003B5001229207904201D1816301E08AB2826311
S31508003B60704701229207904201D1C16301E08AB2EF
S31508003B70C2637047026803231B029A430B891A43E0
S31508003B800260134A904206D001229207904202D060
S31508003B90104A904205D1026870239A438B781A43DB
S31508003BA002600B4A904205D00B4A904202D00B4A5B
S31508003BB0904205D1026B120A12028B7A1A430263EB
S31508003BC04A68C2620A88826201224261704700001E
S31508003BD0002C014000040040004401400048014018
S31508003BE00021C943416000210180018181708172F1
S31508003BF0704710B5FFF7F4FA10BD000070B5FFF76F
S31508003C002BFC05467D21C900FDF784FE0446601E8F
S31508003C100C49884200D90CE0601E0B494861032113
S31508003C20081F00F079FB0020074988610720086112
S31508003C3000BF0420FFF77CFD0021481E00F06CFB46
S31508003C4070BD0000FFFFFF0000E000E010B5022194
S31508003C50154800F07DF8002824D0134800F0C8F86D
S31508003C60C4B21248C078002803D1204600F07CFF71
S31508003C7014E00E48C078022810D10C4800790028B4
S31508003C800CD10B488079AA2804D10948C4710121AE
S31508003C9006480171AA2C01D10548847102210248FF
S31508003CA000F045F810BD000000380140A4030020CC
S31508003CB0F404002010B504462146054800F09CF897
S31508003CC000BF0121024800F03AF80028F9D010BDDB
S31508003CD00038014070B505460E4600247E2000F0E7
S31508003CE09BFA00BF20E0042C19DD701EA04216DDE9
S31508003CF0285D7E2806D17D20FFF7DCFF5E20FFF7D2
S31508003D00D9FF0FE0285D7D2805D1FFF7D3FF5D2099
S31508003D10FFF7D0FF06E0285DFFF7CCFF02E0285D3D
S31508003D20FFF7C8FF601C84B2B442DCDB70BD41619A
S31508003D3070478269520852000A43826170470246F8
S31508003D4090680840002801D0012070470020FCE751
S31508003D500246D0680840002801D00120704700209C
S31508003D60FCE7002A03D003690B43036102E00369F9
S31508003D708B4303617047000070B504460D46002664
S31508003D80E0693021884329790843E061E0694421E4
S31508003D908843A9790843E061E06980088000297AA8
S31508003DA00843E061A0691821884369890843A0612E
S31508003DB0A06904218843297B0843A0610B488442F3
S31508003DC003D1FFF76BFB064602E0FFF755FB0646F5
S31508003DD030462968FDF79EFD0009206230462968AD
S31508003DE0FDF798FD0007000F606270BD00380140BE
S31508003DF001464868C0B27047CAB2026070474B2194
S31508003E00C9010160302101710021817101721821F7
S31508003E10418100210173704710B51C484088030092
S31508003E2000F06BFA0504111E292A2B00174870307A
S31508003E30008CFF211B31884204DA01211348418096
S31508003E4000F00AFA19E011487030008CFF2105319C
S31508003E50884204DA02210D48418000F0FDF90CE0A1
S31508003E600A487030008CFD2804DA0321074841808F
S31508003E7000F0F2F901E000E000BF00BF034890300F
S31508003E804079002801D100F0E7F910BD140300209D
S31508003E9010B530484088002806D0012813D00228DB
S31508003EA020D0032854D12CE080210920C006FEF733
S31508003EB0FCFF01212848FEF7F8FF10210920C0065B
S31508003EC0FEF7F3FF44E001212348FEF7EEFF8021C9
S31508003ED00920C006FEF7E7FF10210920C006FEF7F5
S31508003EE0E2FF35E080210920C006FEF7DEFF01214A
S31508003EF01948FEF7D8FF10210920C006FEF7D3FFA0
S31508003F0026E016494868CD21FDF704FDC007C00F15
S31508003F10002805D080210920C006FEF7C4FF0DE061
S31508003F200E494868CD21FDF7F5FCC007C00F0028EB
S31508003F3004D180210920C006FEF7B7FF01210648F3
S31508003F40FEF7B1FF10210920C006FEF7ACFF00BF3F
S31508003F5000BF10BD1403002000040048C40100205F
S31508003F6010B596488078030000F0C7F90504336C4D
S31508003F70AFFDFC0091482038008CFF2105318842AE
S31508003F8002DB01218D48817040218D48FEF782FFB2
S31508003F9000281DD08B494868FF21F531FDF7BAFC8A
S31508003FA0C007C00F002805D180210920C006FEF7EA
S31508003FB07AFF04E080210920C006FEF776FF10216B
S31508003FC00920C006FEF76FFF01217D48FEF76BFF4B
S31508003FD0F2E07A482038008CFF211B31884202DB48
S31508003FE002217648817040217548FEF753FF002864
S31508003FF027D074494868FF21F531FDF78BFCC007C7
S31508004000C00F002804D101216D48FEF74CFF03E0DC
S3150800401001216B48FEF749FF80210920C006FEF7FB
S3150800402042FF10210920C006FEF73DFF634890387D
S315080040304088012805D0012160489038418000F069
S315080040400BF9B9E05D482038008CFF2125318842FC
S3150800405002DD03215948817040215948FEF71AFFAD
S31508004060002831D057494868FF21F531FDF752FC41
S31508004070C007C00F00280ED180210920C006FEF710
S3150800408014FF01214E48FEF710FF10210920C00633
S31508004090FEF70BFF0DE080210920C006FEF703FF9F
S315080040A010210920C006FEF7FEFE01214448FEF74E
S315080040B0FAFE424890384088002805D000213F483B
S315080040C09038418000F0C8F876E040213C48FEF779
S315080040D0E1FE00284ED0012109030920C006FEF79B
S315080040E0D9FE002811D080210920C006FEF7DDFE82
S315080040F001213348FEF7D9FE10210920C006FEF734
S31508004100D4FE04212D48817026E02E494868FF21F7
S31508004110F531FDF7FFFBC007C00F00280ED180213F
S315080041200920C006FEF7C1FE01212548FEF7BDFE9F
S3150800413010210920C006FEF7B8FE0DE080210920EF
S31508004140C006FEF7B0FE10210920C006FEF7ABFE3A
S3150800415001211B48FEF7A7FE18489038408800281A
S3150800416008D001E027E006E0002114489038418095
S3150800417000F072F820E040211148FEF78BFE002877
S3150800418018D080210920C006FEF78FFE01210C48B1
S31508004190FEF78BFE10210920C006FEF786FE0748AB
S315080041A090384088002805D000210448903841807E
S315080041B000F052F800E000BF00BF10BDA4030020C5
S315080041C000040048C40100200348806840084000F5
S315080041D00149886070470000002C00408021014397
S315080041E0014A116070470000002C004003488068AF
S315080041F0002801D0012070470020FCE7002C004071
S3150800420010B5FFF7F3FF002804D0FFF7DDFF66209F
S3150800421000F002F810BD00004106490E014A11607F
S3150800422070470000002C004004494968FF2281328B
S3150800423091430143014A516070470000002C004039
S3150800424004494968C909C9014206520E1143014A7F
S3150800425051607047002C004010B57E20FFF7DCFF48
S315080042600948FEF7A5FC09490948018205211030CD
S3150800427000F0B3F806491031488140220249044843
S315080042801030FEF7D2FC10BD00900008FBAA000013
S315080042900403002070B505460C460121C802FFF745
S315080042A0BBF8FF208130FFF7BFFF2046FFF7C8FFA6
S315080042B02846FFF793FF70BD10B5024A024900F081
S315080042C07DF810BD454B0008BC0100202021020CDA
S315080042D001D010211046020A01D0104608390209F9
S315080042E001D01046091F820801D01046891E4208CF
S315080042F001D0881E7047081A704730B47446641E89
S315080043002578641CAB4204D3635D5B00E31830BCBC
S3150800431018471D46F8E7000010B5002819DB1A4AA9
S3150800432003231B02D21883089B00D2588307DC0E8E
S31508004330FF23A3409A438B071B0E8407E40EA34072
S315080043401A43114B032424021B198408A4001A518A
S3150800435018E00E4A03071B0F083B9B089B00D25820
S315080043608307DC0EFF23A3409A438B071B0E8407A3
S31508004370E40EA3401A43054B0407240F083CA4087F
S31508004380A4001A5110BD000000E100E01CED00E099
S3150800439002E008C8121F08C1002AFAD17047704700
S315080043A0002001E001C1121F002AFBD1704700005E
S315080043B00149086070470000C0010020F8B516469C
S315080043C00F460446002503E03946B047641C6D1CB9
S315080043D020780028F8D12846F8BD10B502460023F3
S315080043E0002901D1002010BD03E01488921CE018B2
S315080043F083B208464C1EA1B20028F6D11846F2E749
S31508004400F8B50027002600240025F9480079012878
S315080044106FD17E20FFF700FFF648C0790002F54904
S31508004420097A08430746F348467A847A0246D17AD7
S31508004430107B00F0D7FC05460021ED480171EE49D6
S31508004440781A8F426FD01EDCEC49781A8F426BD0EF
S3150800445010DCEB49781A8F4267D006DC442F1CD053
S31508004460E8483818002872D1DEE1882870D08928F3
S31508004470F9D16FE101286CD002286BD003286AD0E5
S315080044800428F0D135E10300FFF737FF0C61C0FAC5
S31508004490F861611926768E415C61062E09D1DA48E3
S315080044A0007800280AD100F041FF0120D64908709B
S315080044B004E0152E02D1012000F038FFCFE1CC48E8
S315080044C02030C078002806D0C9482038028A418A98
S315080044D0002000F085FEC2E1002C0BD1C44820382C
S315080044E0408A00231A46F0210090FE2000F0ADFE17
S315080044F00CE0B5E1012C09D1BD482038008A01231A
S315080045000022F0210090FE2000F09FFEA7E1002C7B
S315080045100CD1BE48408800231A46F3210090FE209D
S3150800452000F093FE0DE05AE056E188E1012C08D12F
S31508004530B648808901230022F3210090FE2000F06E
S3150800454084FE8CE1002C07D1B048458006E085E161
S3150800455014E11DE16AE07AE0AC488581AB488089C0
S31508004560FF21F531884206DA00F0CAFA0022FE2158
S31508004570F42000F09EFE72E1002C09D1A348808841
S3150800458000231A46F1210090FE2000F05EFE0AE0A4
S31508004590012C08D19D48C08901230022F1210090F1
S315080045A0FE2000F052FE5AE1002C02D19748858081
S315080045B003E0012C01D19548C58194488088FF21E4
S315080045C0F53188420ADC9148C089884206DC00F049
S315080045D097FA0022FE21F22000F06BFE3FE1002C44
S315080045E009D18A48C08800231A46E9210090FE208E
S315080045F000F02BFE09E0012C07D119200123002227
S31508004600E9210090FE2000F020FE28E1002C01D1CF
S315080046107E48C580FF202D30854206DA00F070FA04
S315080046200022FE21EA2000F044FE18E1002C0CD1FD
S31508004630764800896421484380B200231A46E2215D
S315080046400090FE2000F001FE00E000BF07E1002C0C
S3150800465006D164212846FDF773F981B26B480181BA
S315080046606A480089FF21F531884206DC00F048FADD
S315080046700022FE21E32000F01CFEF0E01EE0FFE72A
S31508004680002C0CD1614840896421484380B200233C
S315080046901A46EB210090FE2000F0D7FD0DE0012C14
S315080046A00BD15A48008A6421484380B2012300226C
S315080046B0EB210090FE2000F0C8FDD0E0002C07D1C9
S315080046C064212846FDF73CF981B25048418108E04B
S315080046D0012C06D164212846FDF732F981B24B48F0
S315080046E0018200F00DFA0022FE21EC2000F0E1FD27
S315080046F0B5E0012C15D13E4890384088032807DAE2
S3150800470001213B482030C17000204049503948609B
S315080047100022FE21E42000F0CCFD0121344841713D
S3150800472017E0002C10D10021314841712030C170AA
S315080047300022FE21E42000F0BCFD0020324908706A
S3150800474032495039486004E00022FE21E42000F096
S31508004750B0FD84E0002C0FD12648C07A32280CDC44
S315080047602448C17A2948418200F0CAF90022FE216C
S31508004770DF2000F09EFD00E000BF70E02348408A7D
S3150800478000231A46DE210090FE2000F05EFD66E05A
S31508004790002C0FD11748C07A32281CDC1548C17A7C
S315080047A01A48818200F0ACF90022FE21E12000F0CF
S315080047B080FD10E0012C0ED10E48C07A32280ADCA2
S315080047C00C48C17A1148C18200F09AF90022FE21EC
S315080047D0E12000F06EFD42E0002C19D10B48808ADA
S315080047E000231A46E0210090FE2000F02EFD1AE074
S315080047F0A4030020F4040020E9FE0000E0FE000007
S3150800480056FE0000AB01FFFFB8010020140200208D
S31508004810012C08D11348C08A01230022E021009008
S31508004820FE2000F012FD1AE0002C07D101210E48E7
S31508004830C170002202210D48FFF793FA0FE0002C01
S315080048400BD1FF2101310A48FDF7A7F800200849D6
S31508004850891F088002210448C17000E000BF00BF1C
S31508004860F8BD000014020020A4030020003801400F
S31508004870FA040020F0B589B0002008900790069049
S315080048803848007901286BD137488079AA2864D13D
S315080048903548C079322860DA3348C07900285CDDAB
S315080048A03149C97908461938FDF7E8FA0890089891
S315080048B0FDF74AFB04462D4A2D4BFDF7FFF900226A
S315080048C02C4B01910090FDF747F9039102902A4875
S315080048D00068FDF739FB0646039B029AFDF756FA70
S315080048E005910490FDF758FB079024490798FDF7B2
S315080048F0B8F80446FDF7F6FA81B22148018308980C
S31508004900FDF722FB0646194A194BFDF7D7F9044667
S315080049100022184BFDF720F9039102901948006808
S31508004920FDF712FB01910090039B029AFDF72EFA00
S3150800493005910490FDF730FB069010490698FDF79F
S3150800494090F80446FDF7CEFA81B20D48418300F08F
S31508004950D7F800210348C17041710021014801714F
S3150800496009B0F0BDA4030020F4040020091B9E5ED4
S3150800497029CB703F0000F03F5401002000007A4424
S31508004980140200205801002070B505460E4614464C
S31508004990002E02D0012E4AD120E0002D02D0012D92
S315080049A01AD10CE0602101208007FFF74DF800219D
S315080049B001208007FFF7CCF81E4804700CE0602140
S315080049C001208007FFF748F8002101208007FFF73C
S315080049D0C8F81948047000BF00BF28E0002D02D0AF
S315080049E0012D22D110E013480078A0420BD0602197
S315080049F001208007FFF728F8214601208007FFF7E6
S31508004A00A7F80C48047010E00B480078A0420BD0B9
S31508004A10602101208007FFF71FF821460120800743
S31508004A20FFF79FF80448047000BF00BF00BF00BF2F
S31508004A3070BD00006A0100206B01002010B5052436
S31508004A4021E080212C48FCF7A8FF80212A48FDF7A1
S31508004A50D9FF0F212848FFF7C0FC2749C98B884290
S31508004A600CD125481038008A2449884204D000F021
S31508004A70DFF900F045F800E010BD04E0002000E092
S31508004A80401C8028FCDB2046611ECCB20028D8D109
S31508004A9000BF052423E080211748FCF77EFF80210C
S31508004AA01548FDF7CDFF0F211348FFF796FC12496D
S31508004AB0C98B88420ED110481038008A0F4988429F
S31508004AC004D000F0B5F900F01BF802E000F018F881
S31508004AD0D2E704E0002000E0401C8028FCDB2046EA
S31508004AE0611ECCB20028D6D100BF00F0A1F900F0B3
S31508004AF007F800BFC0E7000014020020FBAA000068
S31508004B0010B57E20FFF788FBFEF73CF80B490C48EA
S31508004B1001820F211030FFF760FC09491031C88364
S31508004B20802107481030FDF7C7FF7E20FFF774FB8A
S31508004B30802103481030FDF7CBFF10BDFBAA00000B
S31508004B400402002070B504460D46E1B20548FFF799
S31508004B5053F900BF01210348FFF7F1F80028F9D0FF
S31508004B60204670BD0038014070B5044600257E20F9
S31508004B70FFF752FB98480088FA280ADD0020964974
S31508004B80088096490870FF2101319348801DFCF77B
S31508004B9004FF924800780300FFF7AFFB08052031B1
S31508004BA0425BD5ECFDFC7E2C11D100208A49088099
S31508004BB001208A490870884801880088401C864A6E
S31508004BC01080901D445400201146C87002E0002051
S31508004BD081490880002080490871FBE07E480188E9
S31508004BE00088401C7C4A1080901D445402207B4952
S31508004BF0087010460079001911460871EAE07648EF
S31508004C0001880088401C744A1080901D4454032073
S31508004C107249087010460079001911460871D9E0E2
S31508004C206D4801880088401C6B4A1080901D4454CA
S31508004C3004206A490870104600790019114608715F
S31508004C400846C470C078002802D105206349087058
S31508004C50C0E061484079012856D15E2C1CD15E48D7
S31508004C6000797E305C4908717E215B48028800889D
S31508004C70401C594B1880981D8154801FC078401ECF
S31508004C80C0B21946C870002802DC052053490870CE
S31508004C9000205149487155E05D2C1CD14E480079D9
S31508004CA07D304D4908717D214B4802880088401C9B
S31508004CB0494B1880981D8154801FC078401EC0B289
S31508004CC01946C870002802DC0520444908700020EF
S31508004CD04149487136E04048007900193E49087153
S31508004CE0084601880088401C3B4A1080901D4454A1
S31508004CF0801FC078401EC0B21146C870002821DC4B
S31508004D000520364908701DE07D2C03D10120324963
S31508004D10487117E03048007900192F49087108468C
S31508004D2001880088401C2C4A1080901D4454801F1E
S31508004D30C078401EC0B21146C870002802DC0520A3
S31508004D402649087046E024480079C043401CC5B28D
S31508004D50A54203D106202149087002E007201F4911
S31508004D6008701D4801880088401C1B4A1080901D49
S31508004D7044542FE0184801880088401C164A1080C1
S31508004D80901D44547E2C0BD1012115480171002039
S31508004D90114601E01DE00DE008801049087008E0A2
S31508004DA000200D49088000210D48017100200B499B
S31508004DB008700FE000200949087007480188008834
S31508004DC0401C054A1080901D445400201146088056
S31508004DD000E000BF00BF70BDF4040020B70100204A
S31508004DE0A403002070B50246002013460C461D0297
S31508004DF0FF26360235402543284670BD00BF00BF52
S31508004E0000BF00BF00BF00BF00BF00BF00BFFEE776
S31508004E100549064801820021103041805F218180C2
S31508004E20C180018170470000FBAA0000040300202E
S31508004E3000B5134913480182FF21103041800F2124
S31508004E400181A021C180D22181801E214181AF210B
S31508004E50C1818C210182BE2181810B4901830A49C6
S31508004E6023314183052141820A218182C1820021A1
S31508004E7081830F21FFF7B1FA02491031C88300BDBB
S31508004E80FBAA0000040200205A25000010B57E2067
S31508004E90FFF7C2F95648C07901282AD15448407903
S31508004EA001281CD153494868C821FCF733FDC007BF
S31508004EB0C00F002805D180210920C006FDF7F3FFA1
S31508004EC00DE04C494868C821FCF724FDC007C00F0F
S31508004ED0002804D080210920C006FDF7E6FF10212E
S31508004EE00920C006FDF7DFFF01214348FDF7DBFF78
S31508004EF010BD3F484079012878D13D482030C07818
S31508004F00002802D0012834D10BE040213A48FDF7A9
S31508004F10C1FF002802D1FEF7BBFF01E0FFF720F82A
S31508004F2063E034494868FF21F531FCF7F3FCC00714
S31508004F30C00F00280ED180210920C006FDF7B5FF55
S31508004F4001212D48FDF7B1FF10210920C006FDF704
S31508004F50ACFF0DE080210920C006FDF7A4FF102153
S31508004F600920C006FDF79FFF01212348FDF79BFF97
S31508004F703BE01F482030C078052827D11D494868DE
S31508004F80FF21F531FCF7C6FCC007C00F00280ED17B
S31508004F9080210920C006FDF788FF01211648FDF784
S31508004FA084FF10210920C006FDF77FFF1CE0802141
S31508004FB00920C006FDF777FF10210920C006FDF776
S31508004FC072FF01210C48FDF76EFF0DE080210920D4
S31508004FD0C006FDF76AFF01210748FDF766FF1021A5
S31508004FE00920C006FDF761FF00BF00BF00BF7FE7CD
S31508004FF0A4030020C401002000040048FEF74EFC6C
S31508005000FEF78CF9FDF756FCFDF7F2F90B20FDF7D4
S3150800501021F90C20FDF71EF90920FDF71BF90320DD
S31508005020FDF718F901215648FDF788FA4B200002CA
S31508005030FDF7AAFBFEF7E6F8FEF766FC0D216320EE
S31508005040FEF790FC01214F4841710021C171FFF71D
S31508005050F5FCFEF7D3FD00F09DF8FEF719FF7F215A
S315080050607E20FFF717F98AE04648C07800280AD15B
S31508005070FDF78CFAFFF70AFFFFF7C2F9FEF7F6F815
S3150800508000F06EFF78E03F48C078012836D100234B
S3150800509001221946184600F0A9F900231A461946AE
S315080050A0184600F0A3F9384840683849884204D9B8
S315080050B008213748FDF7F7FE1DE033494868FF2108
S315080050C0F531FCF727FCC007C00F00280ED1802158
S315080050D00920C006FDF7E7FE10210920C006FDF7E6
S315080050E0E2FE01212A48FDF7DEFE04E01021092030
S315080050F0C006FDF7DAFEFDF7F3FA3DE02148C07871
S31508005100022839D1FDF742FAFEF7B0F8002301224A
S315080051101946184600F06AF900231A461946184631
S3150800512000F064F9184840681849884204D90821EB
S315080051301748FDF7B8FE1DE013494868FF21F53109
S31508005140FCF7E8FBC007C00F00280ED18021092014
S31508005150C006FDF7A8FE10210920C006FDF7A3FE2C
S3150800516001210B48FDF79FFE04E010210920C00627
S31508005170FDF79BFEFFF77EFB7E20FFF74DF873E7F2
S3150800518000240140A4030020C4010020204E000092
S315080051900004004810B540210F48FCF7FEFB4021EB
S315080051A00D48FDF76BFC05210B48FFF716F90A4970
S315080051B0498988420AD108481038008A074988422E
S315080051C008D0FFF725FEFFF747F803E0FFF720FEB4
S315080051D0FFF742F810BD000014030020FBAA0000E8
S315080051E0F7B5A0B00C46154680216846FCF7D5FBF6
S315080051F0002700267E2168460170FE214170EF21B6
S3150800520081700721C1702099017100214171847153
S315080052102112C1710121017245722912817201267A
S3150800522005E06846805DC019C7B2701CC6B20B2E71
S31508005230F7DBF843401CC1B26846C1727E21017390
S315080052400D21FEF747FD23B0F0BDFFB585B0054635
S315080052500E460E9F00200190029003900490009045
S3150800526000247E2168460171457186710421C17149
S31508005270079901720899417287723912C17201241D
S3150800528007E001A8015D00980818C0B20090601CEC
S31508005290C4B2082CF5DB0098C043401CC1B268466E
S315080052A001737E2141730A2101A8FEF713FD09B097
S315080052B0F0BDF7B584B005460E4600200090019073
S315080052C002900390002700247E21684601704670EC
S315080052D085700121C170694606980871012405E0A8
S315080052E06846005DC019C7B2601CC4B2052CF7DB5E
S315080052F0F843401CC1B2684641717E21817107217D
S31508005300FEF7E8FC07B0F0BD70B504460D467E20F2
S31508005310FEF782FF03E02078641CFEF7CBFC2846E4
S31508005320691E8DB20028F6D170BD000030B5A1B057
S315080053300446802101A8FCF730FB0025002C02D08A
S31508005340012C20D10FE07E216846017100214171B0
S31508005350442181711321C1711522104902A8FCF755
S3150800536003FB192510E07E2168460171FE21417173
S31508005370442181713321C1713622094902A8FCF7FB
S31508005380F3FA3A2500E000BF00BF802D03DA29466C
S3150800539001A8FFF7B9FF21B030BD00006C0100205D
S315080053A081010020F8B506460C46FCF7EFFE051EFF
S315080053B00F4600D00120014349000B484908411A0D
S315080053C0C90F0DD0002E01D0012100E000210C43A9
S315080053D061004908401AC00F02D10120FEF7E8FF14
S315080053E028463946F8BD00000000F07FFFB58DB0AD
S315080053F005460E46174600200B9000240A90099091
S315080054000890F9480078642803D0F848C07F6428D3
S3150800541003D10121F548017202E00021F348017227
S31508005420002F02D0012F78D128E2F148C089B04276
S3150800543002D1EF48C48A00E00524052C01DC0524C6
S3150800544002E0322C00DB0524301BA8420DDDE748BC
S31508005450C07A00284CD1E64850384068E4495039AB
S3150800546088610121E148C17242E03019A8423FDC57
S31508005470DE48C07A01283BD1DC4820304078012834
S315080054802FD1DB4850384068D94950398969401AC4
S31508005490D84988420DD2D54890380089462820DD5B
S315080054A0D24890380089801E81B2D0489038018150
S315080054B017E0CF4850384068CD4950398969401AB5
S315080054C07D21890188420CD9C848903800895F280F
S315080054D007DAC64890380089801C81B2C3489038DC
S315080054E001810121C1482030417000212038C17254
S315080054F0BE48C07A012875D1301BA84273DDBC4866
S31508005500503840687D21C900884207D26420B649D0
S3150800551008700021B5488173A9E1FDE3B348807B93
S31508005520002869D10121B1488173B148808964286E
S315080055305ADAAE482038018A408B081A81B2AB483D
S31508005540203881830146888BFCF7A3FC0146069028
S31508005550A9480068FCF7C2FA0790FCF7F5FCA74AC9
S3150800556003C2A2492039098C49430846FCF798FC2E
S3150800557007910690A1480CC80698FCF79FFB9F4A1E
S3150800558003C29E4903C9FFF70DFF07910690FCF772
S3150800559003FD9B49086095492039088CFCF779FC7E
S315080055A00146059096480068FCF798FA95490690D2
S315080055B0FCF757FA0790FCF795FC934908700846DC
S315080055C0007864280ADC8C480068FCF7BDFC0022D9
S315080055D08E4B07910690FCF7CBFC08D864208A49C5
S315080055E0087004E040E15BE06420874908707F4862
S315080055F02038018AC1863AE17D485038406C7D21C1
S31508005600C900884247D900207949503948647E48FC
S31508005610007864283BDA75482038018AC08E8142B2
S3150800562030DD0121890774480068FCF7C1F9079045
S31508005630FCF758FC81B26D482038028AC08E101AD1
S31508005640814205DA70480078801E6F4908701EE0AE
S31508005650664920390A8AC98E501AFCF70FFC07904A
S31508005660654801680798FCF7B3FC10D266480078CD
S31508005670801C6549087008460078642807DD6420A0
S31508005680087004E060480078401D5F490870574874
S315080056902038018AC1865C48007853490870E6E0DC
S315080056A0524820304078002875D1514880896428AE
S315080056B003DB64204C490870D9E04D4850384068EF
S315080056C07D21C900884206D2642047490870002116
S315080056D046488173CBE04548807B00285CD1012190
S315080056E0424881734248808964284CDA3F4820380A
S315080056F0018A408B081A81B23C48203881830146CA
S31508005700888BFCF7C6FB014606903B480068FCF709
S31508005710E5F90790FCF718FC384A03C233492039E3
S31508005720098C49430846FCF7BBFB079106903348AA
S315080057300CC80698FCF7C2FA304A03C22F4903C9B7
S31508005740FFF730FE07910690FCF726FC2C49086007
S3150800575026492039088CFCF79CFB01460590284809
S315080057600068FCF7BBF927490690FCF77AF9079019
S31508005770FCF7B8FB2449087008460078642805DD5C
S315080057806420087002E064201F4908701748203812
S31508005790018AC1866BE061E015485038406C7D216E
S315080057A0C900884255D900201149503948640F4824
S315080057B02038018AC08E814243DD012189070E48BF
S315080057C00068FCF7F5F80790FCF78CFB81B20748F0
S315080057D02038028AC08E101A814219DA0A480078DF
S315080057E0801E0949087031E0EA000020A403002061
S315080057F01402002070170000CC000020D000002002
S31508005800D80000200000C842E90000200000F03F50
S31508005810FE490A8AC98E501AFCF730FB0790FC48E5
S3150800582001680798FCF7D4FB10D2FA480078801C68
S31508005830F849087008460078642807DD642008706F
S3150800584004E0F4480078401DF2490870EF48018AE0
S31508005850C186F0480078F049087008E0EB487038CF
S31508005860007AED49087002E00020EB490870EA4822
S31508005870027838461099FFF787F861E3E348403025
S31508005880C078012804D002287ED003287DD194E070
S31508005890E2484088B04202D1E048448A00E00A243F
S315080058A0DE484188408A081AA84209DBDB48503896
S315080058B04068DA49503988620020D94908701AE0E8
S315080058C0D6484088A84216DCD5480078002812D168
S315080058D0CE48018C01870120D1490870CF4850383D
S315080058E04068CE495039896A401ACC49503908620D
S315080058F0084640680863C9488188808A081AA84209
S3150800590009DB0020C7490870C44850384068C349B5
S315080059105039C86217E0C1488088A84213DCC148DC
S31508005920007800280FD1B948018C41870120BD496C
S315080059300870BA4850384068B8495039C96A401A98
S31508005940B64950394862B548503840687D21C90083
S31508005950884228D3AD482030407B002823D1AB4865
S31508005960018C8187012120304173A849888FFCF773
S3150800597090FA01460590AC48FCF7B0F8AB4906909A
S31508005980FCF76FF8079001E00EE01FE0FCF7AAFAB3
S31508005990C1B29E48403001700078642803DB642158
S315080059A09A48403001701AE09C484088B04202D1BB
S315080059B09A48448A00E00A2411E098488088B04250
S315080059C002D19648848A00E00A2408E09348808831
S315080059D0B04202D19148848A00E00A2400BF00BF81
S315080059E0052C01DC052402E0322C00DB3224301BB6
S315080059F0A84219DB89485038406888495039C86137
S31508005A000020486388638148C5832030007B0028CE
S31508005A1005D11E217D48203081770121017300219F
S31508005A207A482030417213E13019A84211DC7748D0
S31508005A302030007B0128F6D10021744820300173FC
S31508005A40FF38E138406875495039C8610020486315
S31508005A50FEE0B542E7DB6D484030C0780128E2D168
S31508005A606A48403080780028DDD16C48408A0A2888
S31508005A700BDB6A495039086AFCF70BFA6C49079040
S31508005A80FCF72CF86B4908601EE06448408A0A282F
S31508005A900FDA6248408A07280BDD60495039086AE0
S31508005AA0FCF7F7F964490790FCF718F861490860AC
S31508005AB00AE05A495039086AFCF7EBF95F4907903A
S31508005AC0FCF70CF85B4908605049088FFCF7E1F9C8
S31508005AD04E490690088FFCF7DCF904905548016892
S31508005AE00498FBF7BEFF05900699FBF7BAFF0790E7
S31508005AF0FCF72AFA524A03C24449088FFCF7E4F92C
S31508005B00039102904E4903C9FFF74CFC019100909E
S31508005B10039B029AFCF73AF900224A4B0591049036
S31508005B20FCF7CCF807910690FCF7F0F981B23748F4
S31508005B307038818039495039486AFCF7AAF93E49D4
S31508005B400790FBF7CBFF3B4908603049488FFCF7C5
S31508005B50A0F92E490690488FFCF79BF90490354822
S31508005B6001680498FBF77DFF05900699FBF779FF16
S31508005B700790FCF7E9F9324A03C22449488FFCF733
S31508005B80A3F9039102902E4903C9FFF70BFC019173
S31508005B900090039B029AFCF7F9F80022294B05911D
S31508005BA00490FCF78BF807910690FCF7AFF981B2E1
S31508005BB016487038C18019488089642823DA17493D
S31508005BC08889FCF766F9154950390690086BFCF781
S31508005BD060F91D490290FBF781FF104904904A8835
S31508005BE00A49098B501AFCF749F903900499FBF7FF
S31508005BF075FF05900699FBF734FF0C490790FBF7EC
S31508005C006DFF03490860012100481FE08403002056
S31508005C10CC000020E9000020EA0000201402002041
S31508005C20DC000020DD000020000082430000C8429E
S31508005C3000803B45C40000200000FA440080BB44B5
S31508005C40E00000200000594000007A44403081708E
S31508005C50BD48007B00287CD001287BD1BA48807FCC
S31508005C60BA490978884207DA0021B748817701736B
S31508005C700020B74988641DE1301BA84210DDB248F0
S31508005C80407B012805D1B048203001782038C177FB
S31508005C9002E06421AC48C1770121AB48017209E1F1
S31508005CA0A9482030C078012804D0022813D0032838
S31508005CB07ED188E03019401BA04208DA3019401B13
S31508005CC0201A5F21081AC1B29F48C17702E05F21F6
S31508005CD09D48C177EDE09E48406B9D49896B401A07
S31508005CE07D21C90088424BD99948406B98498863F9
S31508005CF095482038C08BA84211DD93489038808893
S31508005D000A3081B2904890388180C088642834DB94
S31508005D1064218D48903800E012E1C1802DE08A495F
S31508005D202039C98B691AE20F12195210521C914276
S31508005D3011DA854890388088801C81B2824890386C
S31508005D408180C088642818DB64217F489038C18028
S31508005D5013E0B0E0DCE07C492039C98B691AE20F10
S31508005D6012195210921C914207DD774890388088A4
S31508005D70801E81B274489038818073482038C58364
S31508005D80734840687249C969401A7249884214DDE5
S31508005D906D4890388088401D81B26B489038818064
S31508005DA08088642803DB642167489038818000E096
S31508005DB07BE0674840686649C8616348903801795E
S31508005DC09030C17775E06248406B6149896B401A2B
S31508005DD07D21C900884247D95D48406B5C49886384
S31508005DE059482038C08BA8420FDD57489038C088DC
S31508005DF00A3081B254489038C180C088642830DBA4
S31508005E00642151489038C1802BE04F492039C98B0D
S31508005E10691AE20F12195210521C91420FDA4A48B7
S31508005E209038C088801C81B247489038C180C088A5
S31508005E30642816DB642144489038C18011E0424941
S31508005E402039C98B691AE20F12195210921C914215
S31508005E5007DD3D489038C088801E81B23A489038A0
S31508005E60C18039482038C583394840683849C969E6
S31508005E70401A3949884212DD33489038C088401D97
S31508005E8081B231489038C180C088642803DB642118
S31508005E902D489038C1802E4840682D49C8612A4847
S31508005EA0903881799030C17703E032212648C1774E
S31508005EB000BF00BF30E024482030C078012823D135
S31508005EC03019A8421CDB2048903801799030C177F8
S31508005ED03019801EA8420FDD20480078002816D108
S31508005EE0194890388088401D81B2174890388180BB
S31508005EF001201A4908700AE000201849087006E0CF
S31508005F0000211148C17702E00A210F48C17703E052
S31508005F1000210D48C17700BF00BF0B482030C0786C
S31508005F20012806D10848C27F38461099FEF72CFD8D
S31508005F3005E00548827F38461099FEF725FD00BF23
S31508005F4000BF0B9811B0F0BDA4030020EA000020A2
S31508005F50C401002088130000581B0000E800002038
S31508005F6010B5FE48C078002871D0FC484038408AF1
S31508005F70FF217D31884204DCF8484038008A88428F
S31508005F800ADDF6482038C079002805D1F44948606A
S31508005F900121F2482038C171F148C06BF1498842A5
S31508005FA00AD9EE482038C079002805D1EC4948605E
S31508005FB00121EA482038C171E8482038C07A01280A
S31508005FC01ED1E748C06CE84988421DD90020E4493B
S31508005FD0C864E2484038C18A008A81420BDBDF4840
S31508005FE02038C07900280FD1DD4948600121DB48F7
S31508005FF02038C17108E0D9484038018AC18203E0D7
S31508006000D6484038018AC182D4482038007B012806
S3150800601023D1D348806CD449884222D90020D0495C
S315080060208864CE484038818A408A814210DBCB4852
S315080060302038C079002814D1CCA0FEF73DF90020FD
S31508006040C74948600121C5482038C17109E03BE0CD
S31508006050C2484038418A818203E0C0484038418AB4
S315080060608182BE482038C07901282DD1BB48203806
S315080060704079012828D10023012219461846FFF73E
S31508006080B5F900231A4619461846FFF7AFF9B4487A
S3150800609040687D210901884215D90020B049486029
S315080060A010210920C006FCF7FEFE80210920C00643
S315080060B0FCF7F9FE0121AE48FCF7F5FE0021A748DA
S315080060C020384171C17110BDA44820384079002894
S315080060D063D110210920C006FCF7E5FE80210920BE
S315080060E0C006FCF7E0FE0121A148FCF7DCFE002112
S315080060F09A48C1700023012219461846FFF776F917
S3150800610000231A4619461846FFF770F9944840685E
S31508006110FF21F531884204D220219548FCF7C5FEB7
S3150800612037E220219248FCF7BEFE8D4840688E492A
S315080061308842F5D989482038807A002817D18848B6
S3150800614040687D214901884201D2FDF765FE082194
S315080061508748FCF7A8FE002180482038C171203006
S315080061604170817000207E49086208630BE0402177
S315080061707F48FCF78FFE002805D000217748C170BC
S3150800618001212038417120210920C006FCF78BFE29
S315080061907D20400172494860FBE17048C0780300E1
S315080061A0FEF7ABF806045CB7FFEBEA5B00216B4829
S315080061B04170817000206A49086208630023012241
S315080061C019461846FFF712F900231A4619461846C3
S315080061D0FFF70CF961484038418A01832030C078BE
S315080061E0012809D15E4800696249884203D900211D
S315080061F05A482038C17066E7594840687D21090128
S31508006200884221D900205649486040215848FCF761
S3150800621041FE002809D1FDF7FFFD08215448FCF787
S3150800622042FEFF20F530FCF707FB10210920C006C7
S31508006230FCF739FE80210920C006FCF734FE01214F
S315080062404B48FCF730FE08E020210920C006FCF781
S315080062502CFE08214648FCF728FE99E1404840688C
S31508006260FF21F531884204D220214148FCF71DFE62
S3150800627003E020213E48FCF716FE394948687D218F
S31508006280C900FBF747FB232823D2354948687D21F7
S31508006290C900FBF73FFB19281BD930484038018A4B
S315080062A0FF3871384088814207DA2C484038418ADD
S315080062B0FF387138408881421ADB284880780128DF
S315080062C016D1002026494860C86102212348C170BA
S315080062D00EE0234948687D21C900FBF71BFB2328EC
S315080062E006D300201E494860C86102211B48C170B8
S315080062F01B4A50325188FF327132508A01231A469E
S31508006300FFF774F800231A4619461846FFF76EF881
S315080063103EE113484068FF21F531884204D2202126
S315080063201348FCF7C2FD03E020211148FCF7BBFD2A
S315080063300B484168503000897D22D2005043814283
S3150800634022D2074A50325188FF327132508A0123CD
S315080063501A46FFF74BF800231A4610E0C40300203C
S31508006360C401002070110100B80B0000340D0A00AA
S31508006370000400488813000098E055E011E019462B
S315080063801846FFF733F80BE0002184480173002014
S315080063908349486001218148417203212030C17038
S315080063A0F6E07E482038408AFF217D31884204DCA9
S315080063B07A482038008A88420CDD002301221946D3
S315080063C01846FFF713F800231A4619461846FFF72A
S315080063D00DF828E0724948687D21C900FBF79AFA4A
S315080063E06F4950314989884210D26D4A5032918896
S315080063F0FF327132508A01231A46FEF7F7FF00234F
S315080064001A4619461846FEF7F1FF0CE0634820388D
S31508006410018A418300206249486000215F48017370
S3150800642004212030C170B3E05C482038408AFF213F
S315080064307D31884204DC59482038008A88420CDDC0
S315080064400023012219461846FEF7D0FF00231A46F4
S3150800645019461846FEF7CAFF27E0514948687D21C4
S31508006460C900FBF757FA4E495031098A0F39884255
S3150800647014D24B4A5032D189FF327132108A012325
S315080064800022FEF7B3FF464A5032D188FF327132F6
S31508006490508A01231A46FEF7A9FF06E00020404964
S315080064A0486005213D482030C17071E03C4840688D
S315080064B0FF21F531884204D220213A48FCF7F5FC41
S315080064C00FE037484068FF21F531884209D934483A
S315080064D040684B21C900884203D220213148FCF785
S315080064E0E2FC2F484068304988422DD22B48203894
S315080064F0408AFF217D31884204DC28482038008AFA
S3150800650088420CDD0023012219461846FEF76EFF65
S3150800651000231A4619461846FEF768FF37E0204A50
S315080065205032D189FF327132108A01230022FEF7D8
S315080065305DFF1B4A5032D188FF327132508A0123DF
S315080065401A46FEF753FF22E020211648FCF7ADFC59
S31508006550134840681449C831884218D300201049A6
S31508006560486000210D482030C17020384171002351
S31508006570012219461846FEF739FF00231A4619461E
S315080065801846FEF733FF20210648FCF78CFC00BFAF
S3150800659000BF7E20FDF740FE00BF94E5A40300205F
S315080065A0C401002000040048A4380000CC65000897
S315080065B0C00000200401000090430008D0660008CF
S315080065C0C40100203C080000A043000800000000A9
S315080065D000000000000000000000000000000000AD
S315080065E0000000000000000000000000000000009D
S315080065F0000000000000000000000000000001028A
S3150800660003040102030406070809000000A24A045D
S315080066100000000000000000010203040607080944
S31508006620000000000000000000000000000000005C
S315080066300400000001000000000000000000000047
S31508006640000000000000000000000000000000003C
S31508006650000000000000000000000000000000002C
S31508006660000000000000000000000000000000001C
S31508006670000000000000000000011058594C4C3082
S315080066803131327878787878787878CB7E0001104E
S3150800669058594C4C3031313278787878787878781F
S315080066A004013205054C4C3031310614594132305B
S315080066B0303532384834353034324178787878781D
S315080066C07D5D7E0000000000000000000000000064
S705080018C515
